:100000000C9403070C9447070C9447070C9447077C
:100010000C9447070C9447070C9447070C94470728
:100020000C9447070C9447070C945B120C942D1307
:100030000C9447070C9447070C9447070C94470708
:100040000C9447070C94072C0C9447070C94470713
:100050000C9447070C94FF210C9447070C94470716
:100060000C9447070C9447070C9447070C944707D8
:100070000C9447070C9447070C9447070C944707C8
:100080000C9447070C9447070C9447070C944707B8
:100090000C9447070C9447070C9447070C944707A8
:1000A0000C9447070C9447070C9447079A13BC130A
:1000B000AA14BC13AA1401142414AA1479148C14BD
:1000C000D317D31702180218451883189C1A9C1AC4
:1000D0009C189C1A9D199D19701A9C1A9C1A871AB3
:1000E0000000F0A135002B003171E1000152000049
:1000F0001E00140004001D00E0004D001F001A0047
:1001000016001B0050002A0020000800070006000F
:100110004F002C002100150009001900E2004A00E0
:10012000220017000A00050000004C0001542F00B7
:100130000000E60000004900025430000000E60024
:100140000000290023001C000B00110000006500C6
:10015000240018000D001000E2004B0025000C00E8
:100160000E00360052002800260012000F00370053
:100170005100E3002700130033003800E4004E0074
:100180002E002D003471E500025200000100010034
:1001900001000100010000003A001E0220022202BC
:1001A000010001003B001F022102230201000100A7
:1001B0003C002F0226022F00010001003D0030020A
:1001C00027023000010001003E00310235003502F7
:1001D000000001000100010000000100000001001A
:1001E0000100010000000100000001003F0052007A
:1001F00051002402000001004000240021001E00E4
:10020000270001004100250022001F0027000100F7
:100210004200260023002000370001004300250291
:100220002E0231002E0001004400450001000100B3
:1002300001000000010001000100010001000000B8
:1002400001000100010001000100010001000100A6
:10025000F2000100010001000100F000F1000100C6
:10026000F400010001000100F3000100F5000100AD
:100270000100010001000100000001000100010077
:100280000000010000000100010001000000010069
:100290000000010001000100010001000000010058
:1002A0000100010001000100A9000100010001009E
:1002B0000100AC00AA00B600010001000100AB0083
:1002C000A80001000100010001000100010001007F
:1002D00001000100AE000100010000000A0025300D
:1002E000313662003A200025303258000A722F63FE
:1002F0002030313233343536373839414243444582
:10030000460A000A002530325800626F756E636538
:10031000213A20006C6566742073696465206174FD
:100320007461636865640A006C656674207369644F
:1003300065206E6F7420726573706F6E64696E678E
:100340000A00747279696E6720746F207265736534
:1003500074206D637032333031380A000A444542EC
:1003600055473A20656E61626C65642E0A005B73C6
:100370005D004B6579626F617264207374617274A1
:100380002E0A005B575D005B535D005B525D005BB6
:10039000445D005B435D0016034500720067006F1B
:1003A0000044006F007800200045005A000000164D
:1003B000034500720067006F0044006F0078002062
:1003C0000045005A0000000403090409028D0005DD
:1003D0000100A0FA09040000010301010009211134
:1003E000010001223F000705810308000A090401FA
:1003F000000103010200092111010001224D000743
:1004000005820308000A0904020001030000000934
:1004100021110100012236000705830308000A09A3
:100420000403000203000000092111010001222041
:1004300000070584032000010705040320000109CB
:100440000404000103000000092111010001223908
:1004500000070585031000011201100100000008CB
:10046000EDFE071301000102000105010906A101CB
:10047000050719E029E71500250195087501810296
:100480000508190129059505750191029501750366
:100490009101050719002977150025019578750147
:1004A0008102C00631FF0974A1010975150025FFFD
:1004B0009520750881020976150025FF952075089D
:1004C0009102C005010980A101850216010026B72D
:1004D000001A01002AB700751095018100C0050CB3
:1004E0000901A1018503160100269C021A01002AB8
:1004F0009C02751095018100C005010902A1010946
:1005000001A10005091901290515002501950575A9
:100510000181029501750381010501093009311539
:1005200081257F95027508810609381581257F95FB
:100530000175088106050C0A38021581257F950191
:1005400075088106C0C005010906A101050719E06B
:1005500029E71500250195087501810295017508A7
:10056000810105081901290595057501910295017B
:10057000750391010507190029FF150025FF950650
:1005800075088100C00A002530325820006B65795B
:10059000626F6172645F7265706F72743A20000AF4
:1005A0000025303258006B6579626F6172645F7349
:1005B00065745F6C65643A200064656C5F6B657997
:1005C0005F6269743A2063616E27742064656C3AD7
:1005D00020253032580A006164645F6B65795F6280
:1005E00069743A2063616E2774206164643A20253F
:1005F0003032580A00646F6E652E0A00626F6F67B2
:100600006D61676963207363616E3A202E2E2E2020
:1006100000290A002575002F002575005D2800259A
:10062000640020002564002000256400200025646B
:10063000007C0025303258006D6F7573656B6579ED
:10064000205B62746E7C782079207620685D287249
:1006500065702F61636C293A205B006D6B5F776872
:1006600065656C5F74696D655F746F5F6D6178203F
:100670003D2025640A006D6B5F776865656C5F6D72
:1006800061785F7370656564203D2025640A006DA4
:100690006B5F74696D655F746F5F6D6178203D207D
:1006A00025640A006D6B5F6D61785F7370656564CA
:1006B000203D2025640A006D6B5F696E746572765B
:1006C000616C203D2025640A006D6B5F64656C6180
:1006D00079203D2025640A006D6B5F776865656C45
:1006E0005F74696D655F746F5F6D6178203D202573
:1006F000640A006D6B5F776865656C5F6D61785F3C
:100700007370656564203D2025640A006D6B5F741D
:10071000696D655F746F5F6D6178203D2025640AA7
:10072000006D6B5F6D61785F7370656564203D205F
:1007300025640A006D6B5F696E74657276616C206A
:100740003D2025640A006D6B5F64656C6179203D16
:100750002025640A000A00257500363A207768656E
:10076000656C5F74696D655F746F5F6D61783A2069
:10077000000A00257500353A20776865656C5F6D65
:1007800061785F73706565643A20000A0025750022
:10079000343A2074696D655F746F5F6D61783A20DB
:1007A000000A00257500333A206D61785F7370652B
:1007B00065643A20000A00257500323A20696E749B
:1007C000657276616C286D73293A20000A002575E0
:1007D00000313A2064656C6179282A31306D7329C3
:1007E0003A20000A092D2056616C756573202D0A88
:1007F000004D3E004D25643E20003F00736574208F
:1008000064656661756C740A00433E200077686514
:1008100072652064656C74613A20637572736F72DF
:100820003D25642C20776865656C3D25640A536519
:100830006520687474703A2F2F656E2E77696B6926
:1008400070656469612E6F72672F77696B692F4DD0
:100850006F7573655F6B6579730A000A092D204D0A
:100860006F7573656B6579202D0A4553432F713A77
:1008700009717569740A313A0964656C6179282ACD
:1008800031306D73290A323A09696E746572766186
:100890006C286D73290A333A096D61785F7370654E
:1008A00065640A343A0974696D655F746F5F6D61E0
:1008B000780A353A09776865656C5F6D61785F73B2
:1008C000706565640A363A09776865656C5F7469B6
:1008D0006D655F746F5F6D61780A0A703A097072B6
:1008E000696E742076616C7565730A643A09736584
:1008F000742064656661756C74730A75703A092BAF
:10090000310A646F776E3A092D310A706775703A53
:10091000092B31300A7067646F776E3A092D3130D8
:100920000A0A7370656564203D2064656C746120FB
:100930002A206D61785F7370656564202A202872B3
:100940006570656174202F2074696D655F746F5FD9
:100950006D6178290A003F004D3E2000433E200093
:100960004C25640A000A092D20436F6E736F6C6575
:10097000202D0A4553432F713A09717569740A6D28
:100980003A096D6F7573656B65790A000A092D2048
:100990004D61676963202D0A643A09646562756771
:1009A0000A783A096465627567206D6174726978C6
:1009B0000A6B3A096465627567206B6579626F61DD
:1009C00072640A6D3A096465627567206D6F7573AC
:1009D000650A763A0976657273696F6E0A733A0929
:1009E0007374617475730A633A09636F6E736F6C25
:1009F00065206D6F64650A302D343A096C61796544
:100A000072302D34284631302D4634290A50617514
:100A1000733A09626F6F746C6F616465720A653A4C
:100A200009656570726F6D0A6E3A094E4B524F0A36
:100A30007A3A09736C656570204C4544207465737F
:100A4000740A000A002575002E6E6B726F3A200042
:100A50000A002575002E737761705F6261636B73A6
:100A60006C6173685F6261636B73706163653A2088
:100A7000000A002575002E737761705F67726176DA
:100A8000655F6573633A20000A002575002E6E6F5E
:100A90005F6775693A20000A002575002E7377613B
:100AA000705F72616C745F726775693A20000A004A
:100AB0002575002E737761705F6C616C745F6C6775
:100AC00075693A20000A002575002E636170736C09
:100AD0006F636B5F746F5F636F6E74726F6C3A20DD
:100AE000000A002575002E737761705F636F6E7466
:100AF000726F6C5F636170736C6F636B3A20000A96
:100B00000025303258006B65796D61705F636F6EE0
:100B10006669672E7261773A20000A002575002EFB
:100B20006D6F7573653A20000A002575002E6B65A0
:100B300079626F6172643A20000A002575002E6D9B
:100B400061747269783A20000A002575002E656E7E
:100B500061626C653A20000A0025303258006465F5
:100B60006275675F636F6E6669672E7261773A20A0
:100B7000000A0025750064656661756C745F6C61C0
:100B80007965723A20003F004E4B524F3A206F6613
:100B9000660A004E4B524F3A206F6E0A0074696D20
:100BA00065725F636F756E743A202530346C580A35
:100BB000006B6579626F6172645F6E6B726F3A2071
:100BC00025580A006B6579626F6172645F69646CB5
:100BD000653A2025580A006B6579626F6172645F1F
:100BE00070726F746F636F6C3A2025580A00686FDB
:100BF00073745F6B6579626F6172645F6C65647357
:100C000028293A2025580A000A092D2053746174B6
:100C10007573202D0A004743433A20342E392E3372
:100C2000204156522D4C4942433A20312E382E3124
:100C3000204156525F415243483A20617672350A4C
:100C4000004F5054494F4E533A204C554641204294
:100C50004F4F544D41474943204D4F5553454B4508
:100C6000592045585452414B455920434F4E534FFC
:100C70004C4520434F4D4D414E44204E4B524F204A
:100C80003531320A004255494C443A203230303630
:100C90003038342D6469727479202830313A313615
:100CA0003A3235204A616E203331203230313629D4
:100CB0000A005649443A2030784645454428457252
:100CC000676F446F7820455A29205049443A2030B4
:100CD0007831333037284572676F446F7820455A32
:100CE00029205645523A203078303030310A0044BD
:100CF0004553433A20742E6D2E6B2E206B6579621E
:100D00006F617264206669726D7761726520666FCB
:100D100072204572676F646F780A000A092D2056A9
:100D2000657273696F6E202D0A000A6D6F757365A9
:100D30003A206F66660A000A6D6F7573653A206F18
:100D40006E0A000A6B6579626F6172643A206F66A1
:100D5000660A000A6B6579626F6172643A206F6E91
:100D60000A000A6D61747269783A206F66660A003B
:100D70000A6D61747269783A206F6E0A000A6465C0
:100D80006275673A206F6E0A000A64656275673A99
:100D9000206F66660A000A0A626F6F746C6F616486
:100DA00065722E2E2E2000433E20006565636F6E17
:100DB0006669673A0A00536C656570204C454420AB
:100DC000746573740A000000000000000000000059
:100DD00000010204060A0F17202C3A4A5D71879D14
:100DE000B3C7DAE9F5FCFFFCF5E9DAC7B39D877113
:100DF0005D4A3A2C20170F0A060402010000000089
:100E000000000000000011241FBECFEFDAE0DEBFBB
:100E1000CDBF04B603FE24C08091F9019091FA0180
:100E2000A091FB01B091FC018730904BA740B04BE3
:100E3000B9F41092F9011092FA011092FB0110928C
:100E4000FC0114BE84B7877F84BF88E10FB6F89495
:100E500080936000109260000FBEE0E0FFE3099510
:100E600011E0A0E0B1E0EAEAFBE502C005900D92D6
:100E7000AA33B107D9F711E0AAE3B1E001C01D928E
:100E8000A93FB107E1F70E94930F0C94D32D0C9466
:100E90000000FF93EF93E0913A01F0913B0130970E
:100EA00009F00995EF91FF910895FC01859180303B
:100EB00011F0EFDFFBCF0895FF27E0E230E247FFBC
:100EC0000CC0419597FF09C0EDE260957095809543
:100ED0009095611D711D811D911D27FF02C02195F7
:100EE00030E350E2AA27660F771F881F991FAA1FB9
:100EF000A41710F0A41B63955A95A9F7AA3008F01F
:100F0000A95FA05DAF93F39561157105810591050A
:100F100041F7ED3211F4EF93F395F21718F43F9384
:100F2000F395FBCF8F91B5DFFA95E1F70895E9913D
:100F3000F9918591803021F0853219F0AADFF9CF3F
:100F4000089520E0E89455915532C1F3503311F4DF
:100F5000689455915A3348F4505390F3220F022E5F
:100F6000220F220F200D250FF4CF0EF42195899129
:100F70009991533619F3533729F1533559F1BC017F
:100F800088279927E8945C3621F48991999168948F
:100F90005591543639F446EF7EF077FF0DC08FEF50
:100FA0009FEF0AC055374AE039F0583540E121F04B
:100FB000523642E009F00895FF93EF937DDFEF9101
:100FC000FF91B7CFFF93EF93FC0181918030B9F38C
:100FD00060DFFBCFFF93EF9368DFF1CFDF93CF9319
:100FE000CDB7DEB72596A3DFCF91DF9108956111CC
:100FF0000BC0FC018281882321F085EE0E947016CF
:1010000003C085EE0E94381780E090E008950895AF
:101010006091BC017091BD018091BE019091BF01B2
:101020000E94FE2056985E9825982D9826982E9816
:1010300027982F98813019F0823021F00895259A51
:101040002D9A0895269A2E9A089588E098E0892B83
:1010500011F00E94080880E090E0089556985E988C
:1010600025982D9826982E9827982F988FEF90E006
:10107000909389008093880090938B0080938A00DE
:1010800090938D0080938C00259A2D9A2FEF80E706
:1010900092E0215080409040E1F700C00000269A85
:1010A0002E9A2FEF80E792E0215080409040E1F7A8
:1010B00000C00000279A2F9A2FEF80E792E021507E
:1010C00080409040E1F700C0000025982D982FEF58
:1010D00080E792E0215080409040E1F700C000009E
:1010E00026982E982FEF80E792E021508040904084
:1010F000E1F700C0000027982F9856985E98259831
:101100002D9826982E9827982F98089589EA8093ED
:10111000800089E08093810024982C983F988AB1C0
:101120008F748AB96E98479A8BB1806B8BB9769A17
:101130000E942E0887E098E0892B11F00E94070892
:1011400080E090E0089580E28093000180913C016E
:1011500081110EC00E94F20881E080933C012FEFC4
:1011600083ED90E3215080409040E1F700C0000003
:1011700080E40E94F8088093000181112EC00E9433
:10118000220980930001811128C00E9422098093C6
:101190000001811122C08FE30E9422098093000187
:1011A00081111BC00E941A0980E40E94F8088093F4
:1011B0000001811112C08CE00E942209809300017D
:1011C00081110BC00E94220980930001811105C08A
:1011D0008FE30E942209809300010E941A098091E6
:1011E000000108951092B9008AE08093B800089534
:1011F00094EA9093BC009091BC0097FFFCCF909133
:10120000B900987F983021F0903111F081E0089575
:101210008093BB0084E88093BC008091BC0087FF72
:10122000FCCF8091B900887F883111F0803471F74C
:1012300080E0089584E98093BC008091BC0084FD27
:10124000FCCF08958093BB0084E88093BC0080911C
:10125000BC0087FFFCCF9091B900987F81E0983265
:1012600009F480E0089584E88093BC008091BC007C
:1012700087FFFCCF8091BB00089580910001811110
:1012800015C080E40E94F8088093000181110CC011
:1012900082E10E94220980930001811105C08FEF35
:1012A0000E942209809300010E941A0984B1807F64
:1012B00084B985B1807F85B98AB1837F8AB98BB1C2
:1012C000837F8BB93E98469808950E94A308809327
:1012D00000010E943D0980B38C7080BB81B3836F95
:1012E00081BBAEE3B1E0ECE4F1E08EE08E0F119251
:1012F0001D928E13FCCF86E898E0892B11F00C9498
:10130000860808959F92AF92BF92CF92DF92EF929C
:10131000FF920F931F93CF93DF9380910001882357
:10132000E1F080913D018F5F80933D01811115C0F7
:1013300082E493E00E9455070E94A3088093000175
:10134000882329F088E293E00E94550706C084E1D3
:1013500093E00E9455070E942E080EE311E0C0E0C2
:10136000D0E0BB24B39482E0A82ECC24C394D12C2B
:1013700025E0E22E23E0F22EC730D10500F5809162
:101380000001811164C080E40E94F808809300018C
:10139000811112C082E10E94220980930001811113
:1013A0000BC0C6010C2E01C0880F0A94EAF7809585
:1013B0000E942209809300010E941A0948C0CA3085
:1013C000A1F028F4C83059F0C93061F005C0CC3024
:1013D00089F070F0CD3089F0209A289810C0219AB9
:1013E00029980DC0229A2A980AC0239A2B9807C0E0
:1013F000529A01C0539A5B9802C03E9A469890EA6E
:101400009A95F1F79FB1799902C082E001C080E01E
:1014100091709B25982B7C9902C084E001C080E0EC
:10142000892B7D9902C038E001C030E0832B7E9982
:1014300002C020E101C020E0822B9FB19095991F4E
:101440009927991F9295990F907E892B10C08091B2
:101450000001811174C080E40E94F80880930001AB
:10146000882309F459C0912C0E941A09892DF8018A
:101470009081981739F1808380910101882301F1CF
:101480008091D70180FF04C08AE093E00E94550755
:101490008091D70180FF0CC0809101011F928F9332
:1014A000FF92EF920E94EE070F900F900F900F9017
:1014B0008091D70180FF04C083E093E00E9455072C
:1014C000A09201010E943D0921960F5F1F4FCE306F
:1014D000D10509F051CF809101018823B1F08150ED
:1014E00080930101882339F08FE99FE00197F1F79C
:1014F00000C000000AC0ACE4B1E0EEE3F1E0CF01CF
:10150000825F91919D938E13FCCF85E298E0892BA9
:10151000C1F00E94250815C083E10E942209809332
:1015200000018111A0CF81E40E94F808809300019E
:10153000811199CF0E943309982E909495CF80E025
:1015400096CF81E0DF91CF911F910F91FF90EF90A7
:10155000DF90CF90BF90AF909F900895E82FF0E07C
:10156000E45BFE4F80810895CF92DF92EF92FF926D
:101570000F931F93CF93DF938CEE92E00E94550759
:101580008CE4E82E81E0F82EC0E0D0E097EEC92E82
:1015900092E0D92E0EED12E0DF93CF93DF92CF923F
:1015A0000E94EE0784EE92E00E945507F7018191B8
:1015B0007F0190E00E9464219F938F931F930F936C
:1015C0000E94EE078CED92E00E94550721968DB7A0
:1015D0009EB708960FB6F8949EBF0FBE8DBFCE3053
:1015E000D105D1F6DF91CF911F910F91FF90EF9030
:1015F000DF90CF9008958B3B910578F4883A910560
:1016000040F5853A9105D0F48430910508F0B1C0D9
:101610008130910509F4ADC06BC0803E910508F49E
:1016200067C0883E910508F4A4C09C01205F310981
:101630002031310508F05CC090650895853A910528
:1016400009F459C0863A910509F058C082E890E43F
:101650000895883A910509F454C0893A910509F42E
:1016600053C08A3A910509F452C08B3A910509F4A6
:1016700051C08C3A910509F450C08D3A910509F496
:101680004FC0803B910509F44EC08E3A910509F494
:101690004DC08F3A910509F44CC0813B910509F486
:1016A0004BC0823B910509F44AC0833B910509F484
:1016B00049C0843B910509F448C0853B910509F474
:1016C00047C0863B910509F446C0873B910509F464
:1016D00045C0883B910509F444C0893B910509F454
:1016E00043C08A3B910509F442C080E094E4089528
:1016F00080E090E0089581E890E4089583E890E424
:10170000089582EE94E4089589EE94E408958AEEB3
:1017100094E4089585EB94E4089586EB94E40895A9
:1017200087EB94E408958CEC94E408958DEC94E4B4
:10173000089583E895E408958AE895E4089582E998
:1017400095E4089584E995E4089581E296E4089586
:1017500083E296E4089584E296E4089585E296E4AF
:10176000089586E296E4089587E296E408958AE271
:1017700096E40895089596E0799FF001112494E588
:10178000899FE00DF11D1124E60FF11DEE0FFF1FE3
:10179000EC51FF4F859194910895880F991FFC019A
:1017A000E05AF040859194910895880F991FFC01AB
:1017B000E052FF4F85919491089526E0729FF001C9
:1017C000112444E5849FE00DF11D1124E60FF11D65
:1017D000EE0FFF1FEC51FF4F859194919C013A95BC
:1017E00021154FE1340708F41EC13F512115304146
:1017F00020F49F700E94D50B08959C013053211551
:10180000304118F49927906C0895811520E59207CE
:1018100069F40E94BE1A4FEF84E39CE0415080407F
:101820009040E1F700C000000C942422813020E5B4
:10183000920751F48CE593E00E9455078091D701FF
:1018400081608093D70108959C0130552115304166
:1018500008F051C0292F33272F703327213031054D
:10186000D9F4AC014370552702C0220F331F4A95AB
:10187000E2F73C68AC0164E0440F551F6A95E1F75C
:1018800044275370242B352B73E0880F991F7A95CA
:10189000E1F7807699271DC02230310529F4982F71
:1018A0008827816F906A089523303105A9F4AC012F
:1018B0004370552721E030E002C0220F331F4A95C4
:1018C000E2F73C6843E0880F991F4A95E1F7807E74
:1018D0009770822B932B089524303105E1F4AC01ED
:1018E0004370552721E030E002C0220F331F4A9594
:1018F000E2F73A68E7CF9C0130572115304118F4E0
:101900009F70906208959C0130582115304118F461
:101910009F70906A0895803E9105E0F4803C9105A7
:1019200058F58133910509F46FC048F48932910567
:1019300009F463C08A32910509F46DC072C089331D
:101940009105E9F082389105D1F08533910509F4CC
:101950004DC067C0833E910581F138F4803E91050A
:10196000B9F0823E9105D9F05CC0863E910561F1E7
:10197000873E9105A1F155C00E94CD0B089520919D
:10198000EA0120FD02C021FF4CC080EE90E049C07A
:101990008091EA0180FFF9CF89E390E042C0809115
:1019A000EA0182FF0EC08091EA0184FF03C080E05B
:1019B00090E037C083EE90E034C08091EA0182FF6E
:1019C000F2CF82EE90E02DC08091EA0183FF0BC040
:1019D0008091EA0184FDEBCF87EE90E022C08091F8
:1019E000EA0183FFF5CF86EE90E01BC08091EA010B
:1019F00085FF07C089E290E014C08091EA0185FF6D
:101A0000F9CF85E390E00DC08091EA0186FF07C021
:101A10008AE290E006C08091EA0186FFF9CF81E377
:101A200090E00E94FB0A0895089580916D01089549
:101A30009FB7F89410925C019FBF9091F001943091
:101A400009F057C09091E9009F703091EC00232F6E
:101A5000217030FD20E8922B24E02093E9002091B2
:101A6000EB0020FF43C02091EE0027FF3FC02091F4
:101A70005A01222321F02091E80025FF37C010925F
:101A80005A0126E03091E80035FD15C03091F00193
:101A9000343061F53091EB0035FD28C0215021F440
:101AA00081E080935A0122C0EFE9FFE03197F1F71E
:101AB00000C00000E7CF8093F1008091E80085FD31
:101AC0000AC08091E80080FFFCCF8091E8008E770B
:101AD0008093E80006C08FB7F89421E020935C0162
:101AE0008FBF9F709093E90080E008959F7090935E
:101AF000E9008FEF0895CF93DF9300D01F92CDB709
:101B0000DEB79C018091F001843019F593E0998350
:101B10003B832A839093E9008FEF9091E8008150F6
:101B200095FD06C095ED9A95F1F700008111F5CF6E
:101B30008091E80085FF0DC040E050E063E070E078
:101B4000CE0101960E944B108091E8008E77809321
:101B5000E8000F900F900F90DF91CF910895CF93F1
:101B6000DF9300D01F92CDB7DEB72091F001243073
:101B700021F522E029839B838A8383E08093E90017
:101B80008FEF9091E800815095FD06C095ED9A95F4
:101B9000F1F700008111F5CF8091E80085FF0DC0BD
:101BA00040E050E063E070E0CE0101960E944B10EF
:101BB0008091E8008E778093E8000F900F900F904F
:101BC000DF91CF9108952091F0012430F1F422E0CB
:101BD0002093E9002FEF3091E800215035FD06C039
:101BE00035ED3A95F1F700002111F5CF2091E8008D
:101BF00025FF0BC040E050E065E070E00E944B1014
:101C00008091E8008E778093E8000895CF93DF936A
:101C10002091F001243009F048C0EC0180910C01C2
:101C20008823E1F080910D018823C1F085E0809345
:101C3000E9008FEF9091E800815095FD06C095E195
:101C40009A95F1F700008111F5CF8091E80085FFAA
:101C50002CC040E050E060E170E017C081E080936C
:101C6000E9008FEF9091E800815095FD06C095ED59
:101C70009A95F1F700008111F5CF8091E80085FF7A
:101C800014C040E050E068E070E0CE010E944B10CC
:101C90008091E8008E778093E80080E1FE01ADE559
:101CA000B1E001900D928A95E1F7DF91CF9108950F
:101CB00083E993E00E9455078091EF01811109C0EB
:101CC0000E94E0110E943D128091E20084608093A6
:101CD000E20008958FE893E00E9455071092EF010B
:101CE00008958BE893E00C94550787E893E00E94F1
:101CF00055070C94F42B83E893E00E9455070E944B
:101D0000BA210E94FA2B0E94E2140C94140D209127
:101D10005B012F5F822F62E30E94682D992319F0E7
:101D200020935B01089510925B0180915C018823F0
:101D300071F18091F001843041F58091E9008F705C
:101D40002091EC00922F917020FD90E8892B94E077
:101D50009093E9009091EB0090FF14C09091EE00F9
:101D600097FF10C09091E80095FF03C01092F1001A
:101D7000F9CF9091E80090FF05C09091E8009E7720
:101D80009093E8008F708093E90010925C010895B1
:101D900042E061EC81E00E945A1142E061EC82E095
:101DA0000E945A1142E061EC83E00E945A1142E223
:101DB00061EC84E00E945A1142E161EC85E00C94F0
:101DC0005A118091F201833009F455C030F481300A
:101DD00071F0823009F48EC008958A3009F47AC017
:101DE0008B3009F460C0893009F09CC020C080911C
:101DF000F101813A09F096C08091E800877F8093D5
:101E0000E8008091F5019091F601892B21F460E1C1
:101E10008DE591E003C060E080E090E070E00E941A
:101E200096108091E8008B778093E8000895809168
:101E3000F101813209F076C08091F5019091F601AF
:101E4000009719F0049709F06DC08091E800877F32
:101E50008093E8008091E80082FD05C08091F00148
:101E60008111F8CF5FC08091F10080936D01809166
:101E7000E8008B7753C08091F101813A09F052C09C
:101E80008091F5019091F601892B09F04BC080916A
:101E9000E800877F8093E8008091E80080FFFCCF16
:101EA00080910C0136C08091F1018132D9F5809189
:101EB000F5019091F601892BA9F58091E800877FC3
:101EC0008093E8000E948F118091F30180930C01B0
:101ED0000C94BE1A8091F101813221F58091E800C5
:101EE000877F8093E8000E948F118091F401809396
:101EF0006E0108958091F101813AA1F48091E8008A
:101F0000877F8093E8008091E80080FFFCCF80917C
:101F10006E018093F1008091E8008E778093E80055
:101F20000C948F11089584B7877F84BF88E10FB622
:101F3000F89480936000109260000FBE90E080E8FB
:101F40000FB6F89480936100909361000FBE0E94D9
:101F50006F150E94E0110E943D128091E2008460A2
:101F60008093E20088E19DE00E94F92078940E942D
:101F7000C2140E94711582E091E00E94DD140E945B
:101F8000E22B82E793E00E9455078091F0018530B3
:101F900089F48EE693E00E9455070E947E2180918D
:101FA000EE01882391F30E94A621882371F30E94F9
:101FB0003510EBCF0E949F15E8CF292F3327233010
:101FC0003105C9F064F42130310581F0223031054A
:101FD00009F043C08DE890E02BEC33E042C02132A1
:101FE0003105F1F02232310541F137C082E190E054
:101FF00028E534E036C099278130910541F08230E0
:10200000910541F0892B49F5E7ECF3E005C0EFEAD3
:10201000F3E002C0E7E9F3E0849190E09F0121C082
:102020006530D8F4E62FF0E0EE0FFF1FEB5DFE4FBA
:102030002081318189E090E014C0653070F470E057
:10204000FB01EE0FFF1FE55EFE4F20813181FB019A
:10205000EA5EFE4F808190E004C080E090E020E0E6
:1020600030E0FA0131832083089580E189BD82E167
:1020700089BD09B400FEFDCF8091D8008F7D80938B
:10208000D8008091E00082608093E0008091E000C1
:1020900081FDFCCF0895CF92DF92EF92FF920F93D4
:1020A0001F93CF93DF93EC018B016A010E94AE1165
:1020B000811133C0C114D10439F0F60180819181BE
:1020C000081B190BC80FD91FE12CF12C01151105A4
:1020D00019F18091E80085FD16C08091E8008E77A7
:1020E0008093E800C114D10449F0F6018081918108
:1020F000E80EF91EF182E08285E00FC00E94AE1169
:10210000882321F30AC089918093F10001501109BD
:10211000FFEFEF1AFF0ADACF80E0DF91CF911F9136
:102120000F91FF90EF90DF90CF9008952091F701ED
:102130003091F8012617370748F06115710539F419
:102140002091E8002E772093E80001C0B90140E01B
:1021500061157105A9F12091F001222309F443C012
:10216000253009F442C02091E80023FD40C02091B1
:10217000E80022FD32C02091E80020FFE9CF409125
:10218000F3002091F20030E0342BFC01CF01611507
:10219000710559F02830310540F481918093F100A8
:1021A000615071092F5F3F4FF1CF41E02830310579
:1021B00009F040E02091E8002E772093E800C8CF96
:1021C0004111C9CF0AC08091F001882361F08530A8
:1021D00061F08091E80083FD0AC08091E80082FFF1
:1021E000F2CF80E0089582E0089583E0089581E0D1
:1021F00008952091F7013091F8012617370748F02C
:102200006115710539F42091E8002E772093E800DC
:1022100001C0B901FC0120E06115710591F18091C7
:10222000F001882309F440C0853009F43FC0809153
:10223000E80083FD3DC08091E80082FD2FC08091C1
:10224000E80080FFE9CF2091F3008091F20090E058
:10225000922B6115710559F08830910540F4249155
:102260002093F1003196615071090196F2CF21E07F
:10227000089709F020E08091E8008E778093E800CD
:10228000CBCF2111CCCF0AC08091F001882361F01F
:10229000853061F08091E80083FD0AC08091E800FC
:1022A00082FFF2CF80E0089582E0089583E00895F0
:1022B00081E00895982F973058F59093E90098178A
:1022C00039F07091EC002091ED005091F00003C0C6
:1022D000242F762F50E021FF19C03091EB003E7F74
:1022E0003093EB003091ED003D7F3093ED00309165
:1022F000EB0031603093EB007093EC002093ED0025
:102300005093F0002091EE0027FF07C09F5FD3CFCE
:102310008F708093E90081E0089580E008958091B6
:10232000F10187FF11C08091E80082FD05C0809116
:10233000F0018111F8CF11C08091E8008B770BC0BC
:102340008091F001882349F08091E80080FFF8CF68
:102350008091E8008E778093E80008952091E40052
:102360003091E50095E64091EC00842F817040FFAC
:1023700022C08091E80080FD1CC08091F00188237C
:1023800091F0853091F08091EB0085FD10C0409177
:10239000E4005091E5004217530729F39A01915048
:1023A00011F784E0089582E0089583E0089581E0C4
:1023B000089580E008954091E80042FFDECF08953F
:1023C0000E944E120E945612E0EEF0E08081816081
:1023D0008083E8EDF0E080818F77808319BCA7EDE2
:1023E000B0E08C918E7F8C9380818F7E8083109261
:1023F000EF0108950F931F93CF93DF930E944E1226
:102400000E945612C8EDD0E088818F77888388813A
:102410008068888388818F7D888319BC1092F00141
:102420001092EC011092EE011092ED0100EE10E01E
:10243000F80180818B7F808388818160888342E07E
:1024400060E080E00E945A11E1EEF0E080818E7F32
:102450008083E2EEF0E0808181608083808188600B
:102460008083F80180818E7F80838881806188836A
:10247000DF91CF911F910F910895E8EDF0E08081F9
:102480008F7E8083E7EDF0E080818160808384E04F
:1024900082BF81E08093EF010C94FA11E8EDF0E047
:1024A00080818E7F80831092E20008951092DA007E
:1024B0001092E10008951F920F920FB60F9211240F
:1024C0002F933F934F935F936F937F938F939F933C
:1024D000AF93BF93EF93FF938091E10082FF0BC016
:1024E0008091E20082FF07C08091E1008B7F8093A2
:1024F000E1000E94870E8091DA0080FF1FC080916A
:10250000D80080FF1BC08091DA008E7F8093DA00B4
:102510008091D90080FF0DC080E189BD82E189BD35
:1025200009B400FEFDCF81E08093F0010E94580EB7
:1025300005C019BC1092F0010E946A0E8091E10062
:1025400080FF19C08091E20080FF15C08091E200F9
:102550008E7F8093E2008091E20080618093E200B0
:102560008091D80080628093D80019BC85E0809368
:10257000F0010E94750E8091E10084FF30C08091CF
:10258000E20084FF2CC080E189BD82E189BD09B4ED
:1025900000FEFDCF8091D8008F7D8093D800809180
:1025A000E1008F7E8093E1008091E2008F7E809336
:1025B000E2008091E20081608093E2008091EC0172
:1025C000882311F084E007C08091E30087FD02C0FA
:1025D00081E001C083E08093F0010E947B0E809136
:1025E000E10083FF29C08091E20083FF25C0809134
:1025F000E100877F8093E10082E08093F0011092F8
:10260000EC018091E1008E7F8093E1008091E200F7
:102610008E7F8093E2008091E20080618093E200EF
:1026200042E060E080E00E945A118091F0008860F2
:102630008093F0000E94710EFF91EF91BF91AF91D6
:102640009F918F917F916F915F914F913F912F91CA
:102650000F900FBE0F901F9018951F920F920FB6FC
:102660000F9211242F933F934F935F936F937F9318
:102670008F939F93AF93BF93CF93DF93EF93FF938A
:10268000C091E900CF708091EC00D82FD17080FD0F
:10269000D0E81092E9008091F000877F8093F000ED
:1026A00078940E9471131092E9008091F000886084
:1026B0008093F000CD2BCF70C093E900FF91EF9194
:1026C000DF91CF91BF91AF919F918F917F916F914A
:1026D0005F914F913F912F910F900FBE0F901F90E0
:1026E00018951F93CF93DF93CDB7DEB7AA970FB698
:1026F000F894DEBF0FBECDBFE1EFF1E088E08E0FB2
:102700009091F10091938E13FBCF0E94E10E809186
:10271000E80083FF1FC18091F1019091F201492FE0
:1027200050E04A30510508F015C1FA01EA5AFF4F4E
:102730000C94882D803881F0823809F00BC180918B
:10274000F5018F708093E9008091EB0085FB88276D
:1027500080F91092E90006C08091ED019091EE01A0
:10276000911182609091E800977F9093E8008093A8
:10277000F1001092F100C8C0282F2D7F09F0EAC0A7
:10278000882319F0823061F0E5C08091F301813037
:1027900009F0E0C0933009F080E08093EE012BC097
:1027A0008091F301811127C08091F5018F7009F4A8
:1027B000D1C08093E9002091EB0020FF1CC0933032
:1027C00021F48091EB00806214C09091EB00906145
:1027D0009093EB0021E030E0A90102C0440F551FA7
:1027E0008A95E2F74093EA001092EA008091EB00AC
:1027F00088608093EB001092E9008091E800877F69
:1028000086C08111A7C01091F3011F778091E3006A
:102810008078812B8093E3008091E800877F80930C
:10282000E8000E948F118091E80080FFFCCF80912A
:10283000E30080688093E300111102C082E001C0D0
:1028400083E08093F00186C08058823008F082C017
:102850008091F3019091F4018C3D53E0950779F557
:1028600083E08A838AE289834FB7F894DE01139666
:1028700020E03EE051E2E32FF0E050935700E49176
:1028800020FF03C0E295EF703F5FEF708E2F90E066
:10289000EA3010F0C79601C0C0968D939D932F5FCC
:1028A000243149F74FBF8091E800877F8093E8008B
:1028B0006AE270E0CE0101960E94961014C0AE014B
:1028C0004F5F5F4F6091F5010E94DD0FBC01892BC6
:1028D00009F440C09091E800977F9093E8008981C7
:1028E0009A810E94F9108091E8008B778093E8002C
:1028F00031C0803879F58091E800877F8093E800C7
:102900008091EC018093F1008091E8008E778093B4
:10291000E8000E948F111EC081111CC09091F3012C
:102920009230C0F48091E800877F8093E800909314
:10293000EC010E948F118091EC01811106C0809101
:10294000E30087FD02C081E001C084E08093F001D4
:102950000E94C80E8091E80083FF0AC08091E800C1
:10296000877F8093E8008091EB0080628093EB008A
:10297000AA960FB6F894DEBF0FBECDBFDF91CF9100
:102980001F910895CF938091F0018823A1F0C09109
:10299000E900CF709091EC00892F817090FD80E864
:1029A000C82B1092E9008091E80083FD0E9471130A
:1029B000CF70C093E900CF910895909374018093F4
:1029C00073010895E0917301F0917401309721F043
:1029D0000190F081E02D099480E00895EF92FF923C
:1029E0000F931F93CF93DF93E0917301F0917401E4
:1029F0003097B1F18C010280F381E02D099580912F
:102A0000D70182FF2DC080FF04C08DE895E00E94B1
:102A10005507E80110E187E8E82E85E0F82E80915F
:102A2000D70180FF0BC088811F928F93FF92EF9296
:102A30000E94EE070F900F900F900F90115021966B
:102A40001111EDCF8091D70180FF0AC085E895E094
:102A5000DF91CF911F910F91FF90EF900C9455074C
:102A6000DF91CF911F910F91FF90EF900895E0912A
:102A70007301F0917401309721F00480F581E02D0D
:102A80000994089520917101309172018217930782
:102A900071F09093720180937101E0917301F09154
:102AA0007401309721F00680F781E02D0994089594
:102AB00020916F01309170018217930771F090930C
:102AC000700180936F01E0917301F0917401309770
:102AD00021F00084F185E02D0994089508950C9467
:102AE0006E150E94C0210E9465090C948622CF9326
:102AF000C82F8091D70182FF1EC080FF04C086EAE4
:102B000095E00E9455078091D70180FF0CC01F926D
:102B1000CF9381EA95E09F938F930E94EE070F90E9
:102B20000F900F900F908091D70180FF04C08FE924
:102B300095E00E9455078C2FCF910C94140DCF92E5
:102B4000DF92EF92FF920F931F93CF93DF93CDB756
:102B5000DEB72B970FB6F894DEBF0FBECDBF0E9435
:102B6000820986E7C82E81E0D82E00E010E0E02E32
:102B7000802F0E94AE0AF60141916F01F42EF826D3
:102B8000B1F40F5F1F4F0E30110589F78FEF898366
:102B90008A831B820E94C9218160782F9D838C8348
:102BA00049815A816B818D810E94421640C090916B
:102BB000D70191FF04C08B870E94B40A8B8520E067
:102BC00030E04F2D50E0922FBA01022E02C07595D1
:102BD00067950A94E2F760FF24C02E83EF8221E01C
:102BE00030E0690102C0CC0CDD1C9A95E2F790E060
:102BF0008C219D21892B09F420E028870E94C9217E
:102C00008160782F9A8789874E815F8168858A8560
:102C10000E944216F801EA58FE4F8081C826C08201
:102C200006C02F5F3F4F2630310569F6AACF0E94BC
:102C3000F725109175010E94E2141817A1F00E9467
:102C4000E214809375012B960FB6F894DEBF0FBE89
:102C5000CDBFDF91CF911F910F91FF90EF90DF904B
:102C6000CF900C9477152B960FB6F894DEBF0FBE5D
:102C7000CDBFDF91CF911F910F91FF90EF90DF902B
:102C8000CF900895CF93DF93CDB7DEB72B970FB6D4
:102C9000F894DEBF0FBECDBF4F83588769877A8710
:102CA0008B87DE01119686E0FD0111928A95E9F786
:102CB00085E0FE01379601900D928A95E1F74981F2
:102CC0005A816B817C818D819E810E94581D2B963B
:102CD0000FB6F894DEBF0FBECDBFDF91CF91089540
:102CE000CF93882309F4C2C0C82F823859F40E94B8
:102CF000E21481FDBBC089E30E94F41F0E94D3202F
:102D000089E30CC0833879F40E94E21480FDAEC0E0
:102D100083E50E94F41F0E94D32083E50E94472090
:102D2000CF910C94D320843859F40E94E21482FD90
:102D30009DC087E40E94F41F0E94D32087E4EECF59
:102D40008CEF8C0F813A48F48C2F0E948A2A8111D3
:102D50008DC08C2F0E94F41FE3CF80E28C0F88304F
:102D600048F4C77081E001C0880FCA95EAF70E9455
:102D70009C20D6CF8BE58C0F833078F4C53A29F0B0
:102D8000C63A31F083E890E005C081E890E002C0E7
:102D900082E890E0CF910C94421588E58C0F833146
:102DA00008F064C0C83A39F1C93A41F1CA3A49F168
:102DB000CB3A51F1CC3A59F1CD3A61F1C03B69F1CE
:102DC000CE3A71F1CF3A79F1C13B81F1C23B89F141
:102DD000C33B91F1C43B99F1C53BA1F1C63BA9F1BD
:102DE000C73BB1F1C83BB9F1C93BC1F1CA3BC9F11D
:102DF00080E090E038C082EE90E035C089EE90E04F
:102E000032C08AEE90E02FC085EB90E02CC086EBBC
:102E100090E029C087EB90E026C08CEC90E023C0C6
:102E20008DEC90E020C083E891E01DC08AE891E03D
:102E30001AC082E991E017C084E991E014C081E2F0
:102E400092E011C083E292E00EC084E292E00BC0F7
:102E500085E292E008C086E292E005C087E292E057
:102E600002C08AE292E0CF910C945815CF91089558
:102E7000882309F44BC0823859F40E94E21481FF80
:102E800045C089E30E94F41F0E94D32089E30CC04F
:102E9000833871F40E94E21480FF38C083E50E94F9
:102EA000F41F0E94D32083E50E9447200C94D32076
:102EB000843859F40E94E21482FF28C087E40E94FB
:102EC000F41F0E94D32087E4EFCF9CEF980F913A34
:102ED00058F390E2980F983050F4877091E001C059
:102EE000990F8A95EAF7892F0E94A220DFCF9BE5F0
:102EF000980F933020F480E090E00C944215885AAB
:102F0000833120F480E090E00C94581508958823D4
:102F100021F00E949C200C94D3200895882321F056
:102F20000E94A2200C94D3200895BF92CF92DF92EA
:102F3000EF92FF920F931F93CF93DF9300D000D0B7
:102F400000D0CDB7DEB725E0FC01DE01119601907F
:102F50000D922A95E1F7FC014081318102812581A2
:102F600022952F7063817481672B09F4E5C23F3F7E
:102F700019F44F3F09F4E0C27C0149833A83898107
:102F80009A812E830E94B31F182FB92E0E94B21F60
:102F90000E94791EEB2DE295EF70F0E0E05AFF4FB2
:102FA0002E810C94882D8B2D807F9B2D9F70F92E68
:102FB000882319F0F29480EFF822002349F0FF20D3
:102FC00009F467C28F2D0E94AC200E94D32061C2F9
:102FD000812F0E943817FF2009F4AEC28F2D0E9466
:102FE000B22026960FB6F894DEBF0FBECDBFDF919C
:102FF000CF911F910F91FF90EF90DF90CF90BF90F6
:103000000C94D3203B2D307F8B2D8F70303211F0FC
:103010008295807F112319F0113021F12CC00023FB
:10302000B9F0222309F4A0C1213009F09DC12696F0
:103030000FB6F894DEBF0FBECDBFDF91CF911F91C9
:103040000F91FF90EF90DF90CF90BF900C94BC2039
:10305000222319F0213009F46FC28E830E94BF2011
:103060008E8196C1002321F0223008F065C27CC118
:10307000211162C28DC1002321F0222309F474C101
:1030800008C2222309F484C119C22B2D2695269546
:10309000237030E02115310521F021303105D1F0C8
:1030A0004BC2002321F0812F9B2D937002C080E042
:1030B00090E026960FB6F894DEBF0FBECDBFDF912D
:1030C000CF911F910F91FF90EF90DF90CF90BF9025
:1030D0000C944215002321F0812F9B2D937002C088
:1030E00080E090E026960FB6F894DEBF0FBECDBF0D
:1030F000DF91CF911F910F91FF90EF90DF90CF90D4
:10310000BF900C945815812F002319F00E947D2444
:1031100002C00E94E52426960FB6F894DEBF0FBECB
:10312000CDBFDF91CF911F910F91FF90EF90DF9076
:10313000CF90BF900C946A258B2D837009F07BC0D3
:103140000111FAC1812F829586958770880F880FAB
:10315000912F9F70C92ED12CE12CF12C082E04C088
:10316000CC0CDD1CEE1CFF1C0A94D2F714FF12C01D
:103170004FE050E060E070E004C0440F551F661F50
:10318000771F8A95D2F7CB01BA016095709580952B
:10319000909503C060E070E0CB012B2D269526951D
:1031A0002370422F50E042305105D9F04330510591
:1031B00069F16C297D298E299F294130510551F1F2
:1031C00026960FB6F894DEBF0FBECDBFDF91CF912C
:1031D0001F910F91FF90EF90DF90CF90BF900C94D4
:1031E000A01E6C297D298E299F2926960FB6F8945A
:1031F000DEBF0FBECDBFDF91CF911F910F91FF902A
:10320000EF90DF90CF90BF900C94BC1E0E94A01E48
:10321000C701B60126960FB6F894DEBF0FBECDBF2C
:10322000DF91CF911F910F91FF90EF90DF90CF90A2
:10323000BF900C94841E002319F08B2D817001C067
:103240008695882309F478C1812F829586958770A9
:10325000880F880F912F9F70C92ED12CE12CF12C53
:10326000082E04C0CC0CDD1CEE1CFF1C0A94D2F707
:1032700014FF12C04FE050E060E070E004C0440F63
:10328000551F661F771F8A95D2F7CB01BA0160954B
:1032900070958095909503C060E070E0CB012B2D78
:1032A000269526952370422F50E042305105D9F0E3
:1032B0004330510569F16C297D298E299F294130C0
:1032C000510551F126960FB6F894DEBF0FBECDBF63
:1032D000DF91CF911F910F91FF90EF90DF90CF90F2
:1032E000BF900C947A1F6C297D298E299F292696E0
:1032F0000FB6F894DEBF0FBECDBFDF91CF911F9107
:103300000F91FF90EF90DF90CF90BF900C94961F9D
:103310000E947A1FC701B60126960FB6F894DEBF49
:103320000FBECDBFDF91CF911F910F91FF90EF9016
:10333000DF90CF90BF900C945E1F103FD1F118F436
:10334000103E50F4A1C0123F09F463C008F44CC011
:10335000133F09F473C098C01F708B2D8F71002329
:10336000A1F00E94F71E812F26960FB6F894DEBFBB
:103370000FBECDBFDF91CF911F910F91FF90EF90C6
:10338000DF90CF90BF900C9487170E94181F812F59
:1033900026960FB6F894DEBF0FBECDBFDF91CF915A
:1033A0001F910F91FF90EF90DF90CF90BF900C9402
:1033B0008E170023A9F02111BFC08B2D8F71269687
:1033C0000FB6F894DEBF0FBECDBFDF91CF911F9136
:1033D0000F91FF90EF90DF90CF90BF900C943D1F26
:1033E000223008F0A9C0E9CF0023A9F08B2D8F71FE
:1033F00026960FB6F894DEBF0FBECDBFDF91CF91FA
:103400001F910F91FF90EF90DF90CF90BF900C94A1
:10341000F71E002359F38B2D8F7126960FB6F89463
:10342000DEBF0FBECDBFDF91CF911F910F91FF90F7
:10343000EF90DF90CF90BF900C94181F002399F06D
:103440008B2D8F7126960FB6F894DEBF0FBECDBFC1
:10345000DF91CF911F910F91FF90EF90DF90CF9070
:10346000BF900C94E21E26960FB6F894DEBF0FBEF6
:10347000CDBFDF91CF911F910F91FF90EF90DF9023
:10348000CF90BF900C94D81E0023A9F0222309F4FA
:10349000ADCF812F26960FB6F894DEBF0FBECDBFFD
:1034A000DF91CF911F910F91FF90EF90DF90CF9020
:1034B000BF900C947016222309F4ADCF812F26966D
:1034C0000FB6F894DEBF0FBECDBFDF91CF911F9135
:1034D0000F91FF90EF90DF90CF90BF900C94381732
:1034E0004B2D4F70612FC7010E94F70726960FB62C
:1034F000F894DEBF0FBECDBFDF91CF911F910F912A
:10350000FF90EF90DF90CF90BF900C94FC1D4B2D5F
:103510004F70612FC70126960FB6F894DEBF0FBE1D
:10352000CDBFDF91CF911F910F91FF90EF90DF9072
:10353000CF90BF900C94BA0B26960FB6F894DEBFCE
:103540000FBECDBFDF91CF911F910F91FF90EF90F4
:10355000DF90CF90BF9008950E94B9200E948E20E6
:103560000E94D3200E949D260E946A2580E090E060
:103570000E94421580E090E00C9458150E94A9200A
:103580000C94AC1A0E94B31F292F22952F7030E0A3
:103590002C3031054CF42A3031056CF422503109BD
:1035A0002230310588F407C02C30310549F02F3026
:1035B000310531F009C0803E48F0803F29F406C053
:1035C00093FB882780F9089580E0089581E00895AD
:1035D000CF93DF9300D000D01F92CDB7DEB70F900E
:1035E0000F900F900F900F90DF91CF910895CF9390
:1035F000DF9300D000D000D0CDB7DEB726960FB64F
:10360000F894DEBF0FBECDBFDF91CF9108951F9319
:10361000CF93DF93C091840116E080918501C81794
:1036200099F0D0E01C9FF0011D9FF00D1124EA5786
:10363000FE4F4081518162817381848195810E9416
:10364000F71A2196C770E9CFDF91CF911F910895A6
:103650004091B6015091B7016091B8017091B901E4
:103660008091BA019091BB010C94F71A8091BB0133
:1036700082958F7009F054C08091B801882309F4B5
:103680004FC080918401A09185016091B601709135
:10369000B7014091B9015091BA01B6E08A1709F417
:1036A0003FC090E041155105C1F17F3F11F46F3FDC
:1036B000A1F1B89FF001B99FF00D1124EA57FE4F18
:1036C000218172132AC02081621327C02281211117
:1036D00024C0238134812417350710F42150310987
:1036E000241B350B283C3105C0F42091BB012F7001
:1036F00020612093BB0126E0289FF001299FF00D57
:103700001124E557FE4F80818F708061808386EBA6
:1037100091E00E9495170C94071B01968770BECF0D
:103720000895CF92DF92EF92FF920F931F93CF9362
:10373000DF93CDB7DEB762970FB6F894DEBF0FBE4A
:10374000CDBF8C0185E0F801DE011D9601900D9240
:103750008A95E1F7D8014C9111965C9111971296D8
:103760006C9112971396CD90DC9014973091B6011E
:103770007091B7018091B9019091BA01009709F455
:103780006BC17F3F19F43F3F09F466C1E090B80177
:10379000EE2009F4C0C02091BB01C816D90628F05C
:1037A000F601E81BF90BCF0104C0809590958C0DB4
:1037B0009D1DFF24F394883C910578F0F12C207F27
:1037C00009F0C6C07C2DD98AC88A89890E94E81A66
:1037D00086EB91E00E949517B1C0822F807F09F09F
:1037E00046C0751314C0341312C0611110C02F707D
:1037F00020612093BB010E94281B86EB91E00E9470
:1038000095178091BB01D80115968C932EC0CD28B9
:1038100019F15F3F11F44F3FF9F0F62E61111CC012
:10382000809184012091850136E0821709F45AC005
:1038300090E0389FF001399FF00D1124EA57FE4FB8
:103840007181571306C07081471303C072817111D3
:1038500003C001968770E9CFF62E662309F418C1DC
:103860008091BB0181608093BB01F12C11C1751364
:1038700008C0341306C0611104C08091BB01D80197
:10388000C3C04D875E878D859E856A8B0E94C21A54
:103890006A898823E1F16623D1F12091BB01822F4F
:1038A00082958F7090E0029774F08091B6019091AC
:1038B000B70198878F831986DB86CA862C87CE014D
:1038C00007960E94951786E0F801A6EBB1E00190FB
:1038D0000D928A95E1F70E94361B0E94281BFF2457
:1038E000F394D6C04D875E878D859E850E94B31F59
:1038F000292F22952F7030E0223031050CF0BCC00A
:103900009F7009F0B6C0805E883008F4C1C0C8015D
:103910000E949517E4CFC816D90608F453C0F601E3
:10392000E81BF90BCF01883C910508F450C0F12C3D
:103930007C2DD98AC88A89890E94E81AE6EBF1E0D1
:1039400086E0DF011D928A95E9F70E94281BA0C03E
:10395000751314C0341312C0611110C08091BB01E3
:10396000F8018583C8010E94951786E0E6EBF1E037
:10397000DF011D928A95E9F7FE2C8AC04D875E878C
:103980008D859E856A8B0E94C21A6A89882309F4F4
:10399000BECF662309F4BBCF2091BB01822F829555
:1039A0008F7090E002970CF48ECF8091B6019091C9
:1039B000B7019A8389831B82DD82CC822E83CE015C
:1039C00001967FCF809590958C0D9D1DACCFF62EE6
:1039D000662309F49CCF75132EC034132CC020919C
:1039E000BB0120FD1FC0822F82958F70D9F0D801B6
:1039F00015962C9315978F3049F08F5F982F9295DD
:103A0000907F822F8F70892B15968C93C8010E940E
:103A1000951786E0F801A6EBB1E001900D928A952A
:103A2000E1F793CF86E0F801A6EBB1E001900D92AB
:103A30008A95E1F72DC04D875E878D859E850E9412
:103A4000C21A811140CF8091BB0181608093BB017C
:103A5000C8010E9495171CC0662309F458CF4D87F2
:103A60005E878D859E850E94C21A882309F44FCFF8
:103A70002ACF811148CF0CC0243031050CF047CF3C
:103A80009F7009F440CFF8019581907F09F03BCFFA
:103A90008F2D62960FB6F894DEBF0FBECDBFDF91BB
:103AA000CF911F910F91FF90EF90DF90CF900895ED
:103AB0001F93CF93DF93CDB7DEB72C970FB6F89453
:103AC000DEBF0FBECDBF4F83588769877A878B874C
:103AD0009C87CE0107960E94911B882369F08F81F5
:103AE00098852A853B85232BF1F19F3F09F063C020
:103AF0008F3F09F060C037C086E0FE013796DE01D7
:103B0000119601900D928A95E1F76F817885EA858B
:103B1000FB85309741F17F3F11F46F3F21F12091F8
:103B2000850130E0C9010196877099274091840191
:103B300050E08417950709F447C069837A83FD83B1
:103B4000EC8396E0929FD001939FB00D1124AA5769
:103B5000BE4FFE01319601900D929A95E1F7809348
:103B600085010E94071B16E08091840190918501D8
:103B70008917C1F1189FC00111248A579E4F0E94D6
:103B8000911B882379F1E09184011E9FF00111249B
:103B9000EA57FE4F40815181628173818481958112
:103BA0000E94F71A8091840190E00196877099270E
:103BB00080938401D9CF4F81588569857A858B851B
:103BC0009C850E94F71ACFCF0E94BE1A10928501E1
:103BD00010928401E6EBF1E086E0DF011D928A9508
:103BE000E9F7C1CF2C960FB6F894DEBF0FBECDBF5C
:103BF000DF91CF911F910895EF92FF920F931F9342
:103C0000CF93DF938C01892B09F46CC0F12CEE2447
:103C1000E394E8012196F8018491843740F48430DC
:103C200008F051C0813081F0823019F15BC08537D6
:103C300009F444C0A8F19CE7980F903708F052C0EF
:103C40008F770E94381741C00E5F1F4FFE01C4914D
:103C500080E28C0F883048F4C7708E2D01C0880F29
:103C6000CA95EAF70E94AC2014C08C2F0E947016EF
:103C70002DC00E5F1F4FFE01C49180E28C0F883073
:103C800058F4C7708E2D01C0880FCA95EAF70E94BC
:103C9000B2200E94D3201AC08C2F0E94381716C061
:103CA0000E5F1F4FFE01C491CC2381F08FE99FE08E
:103CB0000197F1F700C00000C150F6CF0E5F1F4F13
:103CC000FE01F49003C00E9470168E018F2D882390
:103CD00009F49FCFEFE9FFE03197F1F700C0000052
:103CE0008150F5CFDF91CF911F910F91FF90EF9011
:103CF000089508956093C0017093C1018093C2013B
:103D00009093C3010C94AC1A0F931F930091C001C0
:103D10001091C1012091C2013091C301DC01CB019E
:103D2000802B912BA22BB32B8093C0019093C101C8
:103D3000A093C201B093C3011F910F910C94AC1AD0
:103D40000F931F930091C0011091C1012091C201F6
:103D50003091C301DC01CB0180239123A223B32343
:103D60008093C0019093C101A093C201B093C3019D
:103D70001F910F910C94AC1A0F931F930091C001E7
:103D80001091C1012091C2013091C301DC01CB012E
:103D900080279127A227B3278093C0019093C10168
:103DA000A093C201B093C3011F910F910C94AC1A60
:103DB0001092BC011092BD011092BE011092BF0181
:103DC0000C94AC1A41E050E060E070E004C0440F95
:103DD000551F661F771F8A95D2F74093BC015093F9
:103DE000BD016093BE017093BF010C94AC1A41E019
:103DF00050E060E070E004C0440F551F661F771F5D
:103E00008A95D2F78091BC019091BD01A091BE012D
:103E1000B091BF01482B592B6A2B7B2B4093BC01DF
:103E20005093BD016093BE017093BF010C94AC1A16
:103E300041E050E060E070E004C0440F551F661F91
:103E4000771F8A95D2F7409550956095709580912F
:103E5000BC019091BD01A091BE01B091BF0148236A
:103E600059236A237B234093BC015093BD01609387
:103E7000BE017093BF010C94AC1A41E050E060E0C9
:103E800070E004C0440F551F661F771F8A95D2F754
:103E90008091BC019091BD01A091BE01B091BF0184
:103EA000482759276A277B274093BC015093BD01BF
:103EB0006093BE017093BF010C94AC1A0F931F93D3
:103EC0000091BC011091BD012091BE013091BF0154
:103ED000DC01CB01802B912BA22BB32B8093BC0157
:103EE0009093BD01A093BE01B093BF011F910F91AC
:103EF0000C94AC1A0F931F930091BC011091BD015B
:103F00002091BE013091BF01DC01CB0180239123C0
:103F1000A223B3238093BC019093BD01A093BE0163
:103F2000B093BF011F910F910C94AC1A0F931F9384
:103F30000091BC011091BD012091BE013091BF01E3
:103F4000DC01CB0180279127A227B3278093BC01F6
:103F50009093BD01A093BE01B093BF011F910F913B
:103F60000C94AC1A0895CF92DF92EF92FF920F93C8
:103F70001F93CF93DF938C01C090C001D090C101FB
:103F8000E090C201F090C3014091BC015091BD018D
:103F90006091BE017091BF01C42AD52AE62AF72A92
:103FA000CFE1D0E0D701C6010C2E04C0B695A7958D
:103FB000979587950A94D2F780FF07C0B8018C2F98
:103FC0000E94DD0B8130910531F4219758F7B8013B
:103FD00080E00E94DD0BDF91CF911F910F91FF9048
:103FE000EF90DF90CF90089590910C01992321F0EC
:103FF00090910D01911109C020910E0130910F0196
:10400000F90132969FEF40E030C0982F9695969533
:1040100096959F30A0F4E0910E01F0910F01E90F09
:10402000F11D877021E030E0A90102C0440F551F47
:104030008A95E2F7CA019181892B81830895909135
:10404000D70190FF23C01F928F9387ED95E09F9338
:104050008F930E94EE070F900F900F900F9008958E
:104060009F3F39F04F5F4E3041F051915813F8CFD8
:104070000DC05111F7CF942FF5CF9F3F39F0F901C3
:10408000E90FF11D97FDFA958283089508959091A7
:104090000C01992321F090910D01911109C02091FB
:1040A0000E0130910F01F9013296205F3F4F30C071
:1040B000982F9695969596959F30A8F4E0910E01CD
:1040C000F0910F01E90FF11D877021E030E0A901A7
:1040D00002C0440F551F8A95E2F7CA01809591816D
:1040E0008923818308959091D70190FF16C01F9274
:1040F0008F9389EB95E09F938F930E94EE070F902B
:104100000F900F900F9008953196E217F30729F062
:1041100090819813F9CF1082F7CF089581E090E055
:10412000E0910E01F0910F01E80FF91F1082019646
:1041300080319105A9F708959091D601892B80933C
:10414000D601089580959091D60189238093D60158
:1041500008951092D60108959091D501892B8093EE
:10416000D501089580959091D50189238093D5013B
:1041700008951092D50108958093C4010895109276
:10418000C401089580910E0190910F01FC013196B8
:104190009C01205F3F4F80E0919191118F5FE2176A
:1041A000F307D1F70895E0910E01F0910F0180918E
:1041B000D6018083E0910E01F0910F0190818091F2
:1041C000D501892B80838091C401882361F0E0911F
:1041D0000E01F0910F019081892B80830E94C220F3
:1041E00081111092C40180910E0190910F010C94E5
:1041F000EE1490933B0180933A010895CF92DF92A1
:10420000EF92FF926C01EE24FF24C114D104E1046B
:10421000F10421F0C701B60120E101C020E0C72E62
:10422000D82EE92EFF24C114D104E104F10419F0C1
:10423000285FC701B6016B017C0154E0F694E79456
:10424000D794C7945A95D1F7C114D104E104F1046D
:1042500019F02C5FC701B6016B017C0142E0F694B6
:10426000E794D794C7944A95D1F7C114D104E104D7
:10427000F10419F02E5FC701B601DC01CB01B69540
:10428000A79597958795892B8A2B8B2B09F02F5F04
:10429000822FFF90EF90DF90CF9008958295982F16
:1042A0009C7C392F36953695282F237344E0249F24
:1042B000C0011124932F982B292F2A7A2695892F14
:1042C0008575880F822B08951F93CF93DF931F92DC
:1042D000CDB7DEB799830E944E21182F9981892F7F
:1042E0000E944E21212F30E0322F2227A901482B96
:1042F000CA010F90DF91CF911F9108958091F00135
:10430000843009F11092D80120E488E190E00FB6E2
:10431000F894A895809360000FBE2093600083B747
:10432000817F846083BF83B7816083BF78948895E1
:1043300083B78E7F83BF88E10FB6F89480936000C7
:10434000109260000FBE089508950895CF930E94C3
:10435000A4210E9482090E94A521C0E08C2F0E9406
:10436000AE0A811104C0CF5FCE30C1F701C081E039
:10437000CF9108950E94BE1A0E94E2140C94140D6D
:1043800082E084BD93E095BD9AEF97BD80936E0067
:1043900008952FB7F8948091D9019091DA01A091F6
:1043A000DB01B091DC012FBF0895CF92DF92EF9235
:1043B000FF920F931F932FB7F8944091D90150911A
:1043C000DA016091DB017091DC012FBF6A017B0192
:1043D000EE24FF248C0120E030E0C016D106E20676
:1043E000F30610F4415051099A01281B390BC901F9
:1043F0001F910F91FF90EF90DF90CF9008951F9243
:104400000F920FB60F9211248F939F93AF93BF9388
:104410008091D9019091DA01A091DB01B091DC018A
:104420000196A11DB11D8093D9019093DA01A0934B
:10443000DB01B093DC01BF91AF919F918F910F9001
:104440000FBE0F901F9018950E94E011F8942FEF67
:1044500087EA91E6215080409040E1F700C00000DB
:1044600087E090EBDC018093F9019093FA01A0932F
:10447000FB01B093FC019CE088E10FB6F894A8958D
:10448000809360000FBE90936000FFCFEF92FF9289
:104490000F931F93CF93DF93D82FC0E08C2F0E94F0
:1044A000AE0A00E010E0E82EF12CC701002E02C099
:1044B000959587950A94E2F780FD06C00F5F1F4F20
:1044C0000630110591F709C0602F7C2F80E00E9413
:1044D000BB0BD813F3CF81E004C0CF5FCE30F1F631
:1044E00080E0DF91CF911F910F91FF90EF900895A1
:1044F000CF93C82F8CE20E944622882321F08C2F74
:10450000CF910C94462280E0CF910895CF930E94E2
:10451000D523811102C00E94BB238CEF95E00E943D
:104520005507C5E6C15049F00E9482098FE39CE916
:104530000197F1F700C00000F5CF85EF95E00E94EC
:10454000550789E20E947822811113C18AE20E94F4
:10455000782281110E94BB2385E00E94782281117C
:104560000E9424220E94E0238093D70187E00E94CA
:1045700078228823A9F18BE10E947822882351F0C8
:104580008091D70181FB222720F991E0922790FBAF
:1045900081F90EC08EE00E947822882361F080911C
:1045A000D70182FB222720F991E0922790FB82F924
:1045B0008093D70115C080E10E9478229091D701A5
:1045C000882341F093FB222720F981E0822780FB9A
:1045D00093F904C0892F809580FB90F99093D701BF
:1045E0008091D7010E94E4230E94F2238093EA0184
:1045F00080EE0E947822882341F08091EA01982F72
:10460000909590FB80F98093EA0189E30E947822DB
:10461000882359F08091EA0181FB222720F991E05B
:10462000922790FB81F98093EA0182EE0E94782222
:10463000882359F08091EA0182FB222720F991E03A
:10464000922790FB82F98093EA0186EE0E947822FD
:10465000882359F08091EA0183FB222720F991E019
:10466000922790FB83F98093EA0183EE0E947822DF
:10467000882359F08091EA0184FB222720F991E0F8
:10468000922790FB84F98093EA0185E30E947822C7
:10469000882359F08091EA0185FB222720F991E0D7
:1046A000922790FB85F98093EA0181E30E947822AA
:1046B000882359F08091EA0186FB222720F991E0B6
:1046C000922790FB86F98093EA0181E10E9478228B
:1046D000882359F08091EA0187FB222720F991E095
:1046E000922790FB87F98093EA018091EA010E946A
:1046F000F6238091EA0187FB882780F980930D01DA
:1047000087E20E947822C82F8EE10E9478228111D0
:10471000C2608FE10E9478228111C46080E20E9411
:1047200078228111C86081E20E9478228111C061E3
:1047300082E20E9478228111C06283E20E94782284
:104740008111C06484E20E947822882311F0C0683D
:1047500002C0CC2329F08C2F0E94ED236C2F03C0C4
:104760000E94E923682F70E080E090E0CF910C94E4
:104770007A1ECF9108956DEE7EEF80E090E00E946A
:10478000BE2D60E082E090E00E94B02D60E083E00A
:1047900090E00E94B02D60E084E090E00E94B02D97
:1047A00060E085E090E00C94B02D80E090E00E9405
:1047B000AA2D21E08D3E9E4F09F020E0822F089522
:1047C00082E090E00C94A22D682F82E090E00C949F
:1047D000B02D83E090E00C94A22D682F83E090E050
:1047E0000C94B02D84E090E00C94A22D682F84E00E
:1047F00090E00C94B02D8091DF0180FF0BC06091A0
:10480000130185E0689FB001112475956795759532
:1048100067952BC081FF09C06091130185E0689FF7
:10482000B00111247595679520C082FF07C0609183
:10483000130185E0689FB001112417C09091E00139
:104840009923D1F060911201961788F720911301F6
:1048500085E0289F90011124929FA001939F500D05
:10486000112470E0CA010E94742D6038710540F473
:104870006115710539F002C065E070E0862F08957A
:104880008FE7089581E008958091DF0180FF08C0DF
:104890006091110170E0759567957595679521C0D8
:1048A00081FF06C06091110170E07595679519C090
:1048B00082FF04C06091110170E010C09091E0018E
:1048C0009923C1F0609110019617A0F78091110112
:1048D000899FC001112470E00E94742D6038710519
:1048E00028F46115710521F0862F08958FE708954A
:1048F00081E0089561E070E0F4CF803F21F40E94F0
:10490000FB23819504C0813F29F40E94FB238093FF
:10491000E3010895823F21F40E94FB23819504C0A6
:10492000833F29F40E94FB238093E2010895893F8D
:1049300019F40E94442405C08A3F31F40E944424A3
:1049400081958093E40108958B3F21F40E944424D3
:10495000819504C08C3F29F40E9444248093E50192
:104960000895843F21F48091E101816017C0853F63
:1049700021F48091E101826011C0863F21F4809191
:10498000E10184600BC0873F21F48091E1018860E0
:1049900005C0883F31F48091E10180618093E1019D
:1049A00008958D3F21F48091DF0181600BC08E3F1F
:1049B00021F48091DF01826005C08F3F29F480914E
:1049C000DF0184608093DF010895803F39F4809196
:1049D000E30187FF6CC01092E30169C0813F29F4B5
:1049E0008091E3011816BCF362C09091E201823F0E
:1049F00029F497FF5CC01092E20159C0833F19F47B
:104A00001916CCF354C0893F41F48091E401181683
:104A10000CF04DC01092E4014AC08A3F29F4809105
:104A2000E40187FF44C0F6CF8B3F39F48091E50164
:104A300087FF3DC01092E5013AC08C3F29F4809178
:104A4000E5011816BCF333C0843F21F48091E101E5
:104A50008E7F17C0853F21F48091E1018D7F11C0C9
:104A6000863F21F48091E1018B7F0BC0873F21F4C9
:104A70008091E101877F05C0883F31F48091E10199
:104A80008F7E8093E10113C08D3F21F48091DF017F
:104A90008E7F0BC08E3F21F48091DF018D7F05C09A
:104AA0008F3F29F48091DF018B7F8093DF0180911C
:104AB000E20181110EC08091E30181110AC0809151
:104AC000E401811106C08091E501811102C01092BC
:104AD000E00108958091D70183FF7EC088E396E0CE
:104AE0000E9455078091E1011F928F9383E396E026
:104AF0009F938F930E94EE0781E396E00E945507F3
:104B00008091E201282F332727FD30953F938F9323
:104B10008EE296E09F938F930E94EE078CE296E0E0
:104B20000E9455078091E301282F332727FD3095F8
:104B30003F938F9389E296E09F938F930E94EE07B5
:104B400087E296E00E9455078091E401282F3327E1
:104B500027FD30953F938F9384E296E09F938F9348
:104B60000E94EE0782E296E00E9455078091E501DF
:104B7000282F332727FD30953F938F938FE196E0C1
:104B80009F938F930E94EE078CE196E00E94550759
:104B90008091E0011F928F9389E196E09F938F931C
:104BA0000E94EE0787E196E00E9455078091DF01A1
:104BB0001F928F9384E196E09F938F930E94EE075C
:104BC00081E196E00E9455078DB79EB74C960FB6CF
:104BD000F8949EBF0FBE8DBF81EE91E00E94371505
:104BE0000E94C9219093DE018093DD0108951F93F7
:104BF000CF93DF938091DD019091DE010E94D5215A
:104C0000AC019091E001992321F02091140130E052
:104C100006C0209115018AE0289F900111244217B7
:104C2000530708F486C08091E201C091E301D0915E
:104C3000E4011091E501811107C0C11176C0D111C5
:104C400074C0111172C075C09F3F19F09F5F90939F
:104C5000E001181624F40E94FB238093E201809166
:104C6000E20187FF05C00E94FB2381958093E2014A
:104C70001C1624F40E94FB238093E3018091E3013E
:104C800087FF05C00E94FB2381958093E30160911B
:104C9000E201662339F1C091E301CC2319F17727B2
:104CA00067FD7095872F972F0E94792C23E333E3BC
:104CB00043E35FE30E94DD2C0E94462C6093E201F7
:104CC0006C2F772767FD7095872F972F0E94792C7F
:104CD00023E333E343E35FE30E94DD2C0E94462C91
:104CE0006093E3011D1624F40E9444248093E401A0
:104CF0008091E40187FF05C00E9444248195809340
:104D0000E401111624F40E9444248093E50180916B
:104D1000E50187FF05C00E94442481958093E50149
:104D2000DF91CF911F910C946A259F3F09F08ECFA0
:104D300096CFDF91CF911F910895E1EEF1E085E0EC
:104D4000DF011D928A95E9F71092E0011092DF01D0
:104D500008958BE598E00E9455071F9281E08F939C
:104D60001F9285E08F938DE098E09F938F930E9430
:104D7000EE070F900F900F900F900F900F900895E7
:104D80008330E9F128F4813061F0823009F108952F
:104D9000853009F462C008F449C0863009F474C053
:104DA000089580911501262F30E0280F311D2F3FE7
:104DB000310524F4680F6093150103C08FEF8093D1
:104DC0001501809115011F928F9386E497E072C0C0
:104DD00080911401262F30E0280F311D2F3F31051F
:104DE00024F4680F6093140103C08FEF80931401C3
:104DF000809114011F928F9384E397E05BC08091B0
:104E00001301262F30E0280F311D2F3F310524F4E8
:104E1000680F6093130103C08FEF8093130180919B
:104E200013011F928F9381E297E044C08091120199
:104E3000262F30E0280F311D2F3F310524F4680F55
:104E40006093120103C08FEF8093120180911201D1
:104E50001F928F938CE097E02DC080911101262F37
:104E600030E0280F311D2F3F310524F4680F609387
:104E7000110103C08FEF80931101809111011F92E6
:104E80008F9383EF96E016C080911001262F30E0BB
:104E9000280F311D2F3F310524F4680F6093100156
:104EA00003C08FEF80931001809110011F928F93A8
:104EB00088ED96E09F938F930E94EE070F900F90DE
:104EC0000F900F900895833081F128F4813059F0CC
:104ED0008230D1F00895853009F449C0B8F18630A8
:104EE00009F456C0089580911501681720F4861BB7
:104EF0008093150102C010921501809115011F9237
:104F00008F9389EC96E054C080911401681720F4C7
:104F1000861B8093140102C0109214018091140129
:104F20001F928F9387EB96E043C08091130168171F
:104F300020F4861B8093130102C01092130180910C
:104F400013011F928F9384EA96E032C08091120180
:104F5000681720F4861B8093120102C01092120180
:104F6000809112011F928F938FE896E021C080916B
:104F70001101681720F4861B8093110102C0109262
:104F80001101809111011F928F9386E796E010C066
:104F900080911001681720F4861B8093100102C0D5
:104FA00010921001809110011F928F938BE596E073
:104FB0009F938F930E94EE070F900F900F900F908A
:104FC0000895CF93C82F1F928F9380E699E09F9307
:104FD0008F930E94EE0781E090E0A0E0B0E0BC017A
:104FE000CD0104C0660F771F881F991FCA95D2F79D
:104FF0000E947A1E0F900F900F900F90CF910C94FB
:10500000BE1ACF938D3109F465C0B0F58E3009F426
:10501000CCC100F5873009F49BC1A8F4863009F0B3
:105020006DC28091D701817F8E7F8093D70185E605
:1050300099E00E94550787EA9DE00E94550781E0AC
:105040008093E70180C1883009F44FC08B3009F4A8
:105050007CC154C2863109F4F0C138F4803109F4BE
:10506000B8C1813109F430C249C2893109F4CEC1D5
:105070008B3109F486C142C2853309F437C248F442
:10508000873209F433C208F433C2893209F42EC2DC
:1050900035C2833438F48A3308F02CC2883309F4DB
:1050A00054C12CC2833409F421C2883409F026C2C9
:1050B0000E94BE1A86E99DE00E9455079FEF23EDEE
:1050C00080E3915020408040E1F700C000000E9442
:1050D000242239C186EB9DE00E9455070E94002CD6
:1050E0000E94E2140E94140D2EC18BEA9DE00E94E2
:1050F000550786E79BE00E9455070E94E9231F920F
:105100008F9383E79BE09F938F930E94EE0781E745
:105110009BE00E9455070E94E023C82F8EE59BE08C
:105120000E9455071F92CF9389E59BE09F938F9331
:105130000E94EE0787E59BE00E9455078DE49BE007
:105140000E9455078C2F81701F928F938AE49BE0F9
:105150009F938F930E94EE0788E49BE00E9455077F
:105160008EE39BE00E945507C1FB882780F91F92C0
:105170008F938BE39BE09F938F930E94EE0789E3CD
:105180009BE00E9455078DE29BE00E945507C2FB01
:10519000882780F91F928F938AE29BE09F938F93D9
:1051A0000E94EE0788E29BE00E9455078FE19BE09A
:1051B0000E945507C3FBCC27C0F91F92CF938CE107
:1051C0009BE09F938F930E94EE078AE19BE00E94F1
:1051D00055070E94F223C82F86E09BE00E945507E6
:1051E0001F92CF9381E09BE09F938F930E94EE07E5
:1051F0008FEF9AE00E94550786EE9AE00E945507CD
:105200008C2F81701F928F9383EE9AE09F938F93E0
:105210000E94EE078DB79EB780960FB6F8949EBF9A
:105220000FBE8DBF81EE9AE00E9455078AEC9AE08E
:105230000E945507C1FB882780F91F928F9387EC46
:105240009AE09F938F930E94EE0785EC9AE00E946C
:10525000550783EB9AE00E945507C2FB882780F927
:105260001F928F9380EB9AE09F938F930E94EE079B
:105270008EEA9AE00E9455078CE99AE00E94550751
:10528000C3FB882780F91F928F9389E99AE09F9347
:105290008F930E94EE0787E99AE00E9455078DE8F8
:1052A0009AE00E945507C4FB882780F91F928F93CC
:1052B0008AE89AE09F938F930E94EE0788E89AE02D
:1052C0000E94550786E79AE00E945507C5FB88278C
:1052D00080F91F928F9383E79AE09F938F930E94A8
:1052E000EE0781E79AE00E94550785E59AE00E9463
:1052F0005507C6FB882780F91F928F9382E59AE0B5
:105300009F938F930E94EE0780E59AE00E945507D5
:1053100088E49AE00E945507C7FBCC27C0F91F928A
:10532000CF9385E49AE09F938F930E94EE0783E4E6
:105330009AE00E9455078DB79EB74C960FB6F89429
:105340009EBF0FBE8DBFC1E0DEC08CE899E05BC0A0
:105350008091D701C82FC17080FF09C089E89DE006
:105360000E9455078091D701817F8E7F47C08DE7CE
:105370009DE00E9455078091D70181608093D701FD
:10538000E2CF9091D70191FBCC27C0F981E0C827EB
:10539000892FC0FB81F98093D701CC2319F080E7D6
:1053A0009DE027C082E69DE02EC09091D70192FB40
:1053B000CC27C0F981E0C827892FC0FB82F98093F0
:1053C000D701CC2319F083E59DE013C083E49DE071
:1053D0001AC09091D70193FBCC27C0F981E0C82770
:1053E000892FC0FB83F98093D701CC2351F087E349
:1053F0009DE00E9455078091D70181608093D7017D
:1054000082C08AE29DE00E9455079DCF8BE19DE01E
:105410000E9455078FEE9CE00E94550782EB9CE0AE
:105420000E94550785E89CE00E94550781E49CE0B6
:105430000E94550786E19CE0E6CF88E09CE00E9450
:1054400055070E94E2141F928F938EEE9BE09F936C
:105450008F930E94EE0780910C011F928F9387ED2E
:105460009BE09F938F930E94EE0780916E011F92A5
:105470008F9384EC9BE09F938F930E94EE07809123
:105480000D011F928F9381EB9BE09F938F930E945E
:10549000EE078091D9019091DA01A091DB01B091E2
:1054A000DC01BF93AF939F938F938DE99BE09F9314
:1054B0008F930E94EE078DB79EB746960FB6F8946D
:1054C0009EBF0FBE8DBF3FCF0E94BE1AC0910D017F
:1054D00081E0C827C0930D01CC2329F083E99BE02C
:1054E0000E94550710C088E89BE08DCF80E003C084
:1054F0008D5101C089530E94E12725CF86E89BE0AA
:105500000E945507C0E08C2FCF91089580E0089548
:1055100080E00895CF93C82F8091E701813081F01A
:1055200020F0823009F44FC045C1E0910E01F091A6
:105530000F018081813169F0823209F03DC109C0DB
:10554000E0910E01F0910F018081813111F08232E2
:1055500061F48C2F0E94862A811104C08C2F0E9436
:1055600001282FC081E090E02CC08C2F0E94882A57
:10557000811126C0C431E1F070F4CB3081F0C0312C
:10558000D1F40E94A92688E599E00E94550782E09F
:105590008093E70115C0C93259F0C83361F485E63C
:1055A00099E00E9455078CE599E00E94550708C0D4
:1055B0001092E70103C186E599E00E945507FEC0FD
:1055C00081E08170FDC0C43220F5CE3108F0C0C04A
:1055D000CB3099F1C8F4C73009F0D2C08AE080938B
:1055E000150194E19093140193E09093130180933B
:1055F000120188E08093110188E2809310018CEF02
:1056000097E00E945507BFC0C33149F1C431C1F0D2
:10561000B7C0CB3409F4A9C028F4C93289F0C83323
:1056200061F0AEC0C13509F49EC0C23509F499C01D
:10563000CE3409F0A5C06AE09EC00E94A926A3C08E
:105640008091E601882319F01092E6019CC089E060
:1056500098E00E94550781E08093E701B1C083EE96
:1056600097E00E94550781ED97E00E9455078091D1
:1056700015011F928F938EEC97E09F938F930E945A
:10568000EE078CEC97E00E9455078AEB97E00E94AA
:105690005507809114011F928F9387EB97E09F939A
:1056A0008F930E94EE0785EB97E00E94550786EAEC
:1056B00097E00E945507809113011F928F9383EA10
:1056C00097E09F938F930E94EE0781EA97E00E94F4
:1056D000550780E997E00E945507809112011F92BB
:1056E0008F938DE897E09F938F930E94EE078BE84E
:1056F00097E00E94550786E797E00E945507809142
:1057000011011F928F9383E797E09F938F930E94DD
:10571000EE0781E797E00E9455078AE597E00E942F
:105720005507809110011F928F9387E597E09F9313
:105730008F930E94EE0785E597E00E9455078DB78D
:105740009EB748960FB6F8949EBF0FBE8DBF1BC084
:10575000CE51EC2FF0E0E15DFE4F80818093E601B9
:1057600012C061E003C061E006C06AE08091E6011A
:105770000E94C02608C08091E6010E94632703C0F2
:105780008AEF97E013C08091E601882369F01F92A9
:105790008F9384EF97E09F938F930E94EE070F9073
:1057A0000F900F900F9004C081EF97E00E94550773
:1057B00081E006C01092E70180E002C080E001CFE6
:1057C000CF910895E1E8F0E0808188608083808156
:1057D000816080838FB7F89493E09093890090ED77
:1057E000909388008FBF0895EFE6F0E0808182609B
:1057F00080830895EFE6F0E080818D7F80830895B7
:10580000EFE6F0E0908182E08927808308951F927F
:105810000F920FB60F9211242F933F934F935F93E4
:105820006F937F938F939F93AF93BF93EF93FF9368
:105830008091E8019091E90101969093E9018093AC
:10584000E801811103C082E00E94140DE091E9019A
:10585000E695E695F0E0EA53F24FE4918091E80195
:105860008E1303C080E00E94140DFF91EF91BF9151
:10587000AF919F918F917F916F915F914F913F91E8
:105880002F910F900FBE0F901F90189504D0689421
:10589000B1118DC0089570D088F09F5790F0B92F46
:1058A0009927B751A0F0D1F0660F771F881F991F75
:1058B0001AF0BA95C9F712C0B13081F077D0B1E0D3
:1058C000089574C0672F782F8827B85F39F0B93FE3
:1058D000CCF3869577956795B395D9F73EF4909577
:1058E0008095709561957F4F8F4F9F4F0895E894F5
:1058F00009C097FB3EF490958095709561957F4F18
:105900008F4F9F4F9923A9F0F92F96E9BB279395C5
:10591000F695879577956795B795F111F8CFFAF4D5
:10592000BB0F11F460FF1BC06F5F7F4F8F4F9F4F06
:1059300016C0882311F096E911C0772321F09EE864
:10594000872F762F05C0662371F096E8862F70E0CA
:1059500060E02AF09A95660F771F881FDAF7880FA4
:105960009695879597F9089557FD9058440F551FC0
:1059700059F05F3F71F04795880F97FB991F61F0D1
:105980009F3F79F087950895121613061406551F48
:10599000F2CF4695F1DF08C0161617061806991FB4
:1059A000F1CF86957105610508940895E894BB27A9
:1059B00066277727CB0197F908950BD078C069D077
:1059C00028F06ED018F0952309F05AC05FC011245A
:1059D000EECFCADFA0F3959FD1F3950F50E0551F8E
:1059E000629FF001729FBB27F00DB11D639FAA2734
:1059F000F00DB11DAA1F649F6627B00DA11D661F83
:105A0000829F2227B00DA11D621F739FB00DA11DA3
:105A1000621F839FA00D611D221F749F3327A00D5D
:105A2000611D231F849F600D211D822F762F6A2FF9
:105A300011249F5750408AF0E1F088234AF0EE0F7E
:105A4000FF1FBB1F661F771F881F91505040A9F78B
:105A50009E3F510570F014C0AACF5F3FECF3983E13
:105A6000DCF3869577956795B795F795E7959F5FF2
:105A7000C1F7FE2B880F911D9695879597F908958C
:105A800097F99F6780E870E060E008959FEF80ECF1
:105A9000089500240A941616170618060906089594
:105AA00000240A9412161306140605060895092EFA
:105AB0000394000C11F4882352F0BB0F40F4BF2B69
:105AC00011F460FF04C06F5F7F4F8F4F9F4F0895A9
:105AD000991B79E004C0991F961708F0961B881F40
:105AE0007A95C9F78095089597FB072E16F40094D0
:105AF00007D077FD09D00E948E2D07FC05D03EF41B
:105B0000909581959F4F0895709561957F4F089569
:105B1000EE0FFF1F0590F491E02D0994AA1BBB1B0B
:105B200051E107C0AA1FBB1FA617B70710F0A61B9D
:105B3000B70B881F991F5A95A9F780959095BC01BE
:105B4000CD010895F999FECF92BD81BDF89A9927AC
:105B500080B50895A8E1B0E042E050E00C94C52D76
:105B6000262FF999FECF1FBA92BD81BD20BD0FB679
:105B7000F894FA9AF99A0FBE019608950E94B02DF2
:105B8000272F0C94B12DDC01CB01FC01F999FECF3C
:105B900006C0F2BDE1BDF89A319600B40D924150B5
:0A5BA0005040B8F70895F894FFCFC5
:105BAA002002150D060EE30DAF0D7B0D0101C50197
:105BBA0028080A03140A3F4D3620394605F904C35A
:105BCA0004A3046A04DD03F6030F0428044804014D
:0A5BDA000203040506070809000095
:00000001FF
